:100000000C940B030C9433030C9433030C943303C0
:100010000C9433030C9433030C9433030C94330388
:100020000C9433030C9433030C94580B0C94C70BAF
:100030000C9433030C9433030C9433030C94330368
:100040000C9433030C9433030C9433030C94330358
:100050000C9433030C9433030C9433030C940E0B65
:100060000C9433030C9433030C9433030C94330338
:100070000C9433030C9433030C9433030C94330328
:100080000C9433030C9433030C9433030C94330318
:100090000C9433030C9433030C9433030C94330308
:1000A0000C9433030C9433030C9433034C205348C7
:1000B0004946542B48004C2053484946542B47008E
:1000C0004C2053484946542B46004C20534849463F
:1000D000542B45004C2053484946542B44004C2097
:1000E00053484946542B43004C2053484946542B0F
:1000F00042004C2053484946542B41004E6F206D1E
:100100006F6469666965722B5A004E6F206D6F646B
:1001100069666965722B59004E6F206D6F64696660
:100120006965722B58004E6F206D6F646966696552
:10013000722B57004E6F206D6F6469666965722B74
:1001400056004E6F206D6F6469666965722B5500AD
:100150004E6F206D6F6469666965722B54004E6F37
:10016000206D6F6469666965722B53004E6F206D58
:100170006F6469666965722B52004E6F206D6F6403
:1001800069666965722B51004E6F206D6F646966F8
:100190006965722B50004E6F206D6F6469666965EA
:1001A000722B4F004E6F206D6F6469666965722B0C
:1001B0004E004E6F206D6F6469666965722B4D004D
:1001C0004E6F206D6F6469666965722B4C004E6FCF
:1001D000206D6F6469666965722B4B004E6F206DF0
:1001E0006F6469666965722B4A004E6F206D6F649B
:1001F00069666965722B49004E6F206D6F64696690
:100200006965722B48004E6F206D6F646966696581
:10021000722B47004E6F206D6F6469666965722BA3
:1002200046004E6F206D6F6469666965722B4500EC
:100230004E6F206D6F6469666965722B44004E6F66
:10024000206D6F6469666965722B43004E6F206D87
:100250006F6469666965722B42004E6F206D6F6432
:1002600069666965722B41004C5F4354524C2B4CBC
:100270005F53484946542B44454C455445004C5F18
:100280004354524C2B4C5F53484946542B494E53D0
:10029000455254004C5F4354524C2B4C5F534849D9
:1002A00046542B4F004C5F4354524C2B4C5F5348E9
:1002B0004946542B50004C5F4354524C2B4C5F53D7
:1002C000484946542B454E44004C5F4354524C2BF6
:1002D0004C5F53484946542B484F4D4500534849BD
:1002E0004654320053484946543100535741500058
:1002F000465245512D450056532D4500414C542D35
:1003000045004844472D45004941532D450043527F
:10031000532D450041505052004C4F43004C530068
:10032000464400565300414C54004844470049415C
:10033000530043535200412F5448520046524551F6
:1003400000565300414C5400484447004941530073
:100350004353520000000000000000002A2B280038
:10036000000000000000000000000000000000008D
:10037000000000002C9EB4A0A1A2A434A6A7A5AEA4
:10038000362D3738271E1F20212223242526B3335C
:10039000B62EB7B89F8485868788898A8B8C8D8E88
:1003A0008F909192939495969798999A9B9C9D2F54
:1003B0003130A3AD350405060708090A0B0C0D0EF4
:1003C0000F101112131415161718191A1B1C1DAF34
:1003D000B1B0B500000000002300260029002C0069
:1003E0002F00C902B602A50294027E0268025A02D8
:1003F0004C023E023002220214020602F801EA0117
:10040000DC01CE01C001B201A401960188017A018C
:100410006C015E01500142013401260118010A01FC
:10042000FC00F200E800DE00D400CA00C000B60004
:10043000AC000268206901360131012F013001341E
:1004400001390433043504360431502F5030503410
:1004500050395033503550365031042F0430043465
:1004600004391033103510361031102F103010347D
:1004700010394033403540364031402F4030403411
:100480004039080B000202020000090400000102CA
:1004900002000005240010010524010101042402CA
:1004A0000605240600010705810310004009040128
:1004B00000020A0000000705020240000007058351
:1004C000024000000403090412010002EF0201408F
:1004D0005623518000010102030141584149520055
:1004E0004D4941502058424F5800360332032E03E5
:1004F0002A032603230320031D03190314030E03F9
:1005000008030203FC02F702F002EB02E402DD0240
:1005100009190A1A0B1B0C1C0D1D0E1E101F112091
:10052000122113222100241517161A171D1808006E
:100530001400160015000B02010C04031506051F1C
:100540000807290A09330C0B3D0E0D3E100F3F1210
:100550001140141350034C034803440341033C036C
:100560001F202223252618191B1C1E07000000002F
:10057000240027002A002D00300000000000250084
:1005800028002B002E003100040404040403040599
:100590000202020204030202020206060606060620
:1005A0000404020202040404080201104080401006
:1005B0002040804080080204018040201002011089
:1005C0008010204040200000000200090F000003BE
:1005D0000401000C0000000000000000000000000A
:1005E000000000000005010906A1018502050719A8
:1005F000E029E7150025017501950881029501752F
:10060000088103950675081500257305071900294B
:10061000738100C0F90D11241FBECFEFDAE0DEBFF9
:10062000CDBF15E0A0E0B1E0EAE1F9E202C005903B
:100630000D92AC34B107D9F726E0ACE4B5E001C0C7
:100640001D92A239B207E1F713E0CBE0D3E004C07A
:100650002197FE010E946A11CA30D107C9F70E9492
:100660008B0E0C948B140C940000CF93DF93FC0141
:10067000818190916306482F490F5527551F4830B7
:1006800051059CF5A281B381109709F52FE536E05D
:1006900033832283208120936106809362068091B8
:1006A0006406820F808320916506A22FB0916606B2
:1006B0008A2F821B8917E8F481813D91C82FD0E0F1
:1006C000C45DDB4F38838F5F8183F2CFD9011896E9
:1006D0002D913C91199721153105C1F72FE536E091
:1006E00019963C932E931897D5CF80E0DF91CF9148
:1006F000089581E0FBCFFC0180910E06882311F163
:100700003FB7F89482E08093E9002091F200822FB5
:1007100090E01816190614F481E090E0882339F06F
:10072000289844E640930D064091F100408322232F
:1007300039F02091F200211103C02BE62093E8004C
:100740003FBF08958FEF9FEF089581508F3008F0DD
:1007500047C0E82FF0E0E155FC4F0C946A11CC0340
:10076000D003BE03C403C803F003F003F003D303B4
:10077000D903DD03E103E703F003EB03809180007D
:100780008F77809380000895809180008F7DF9CFCE
:1007900080918000877FF5CF84B58F7784BD0895E1
:1007A00084B58F7DFBCF809190008F7780939000F0
:1007B0000895809190008F7DF9CF80919000877F80
:1007C000F5CF8091C0008F778093C000089580910D
:1007D000C0008F7DF9CF8091C200877F8093C200D7
:1007E00008951F93CF93DF93282F30E0F901EA5348
:1007F000FA4F8491F901E955FA4FD491F901E8577C
:10080000FA4FC491CC23A9F0162F81110E94A503A1
:10081000EC2FF0E0EE0FFF1FE658FA4FA591B491D0
:100820008FB7F894EC91111108C0D095DE23DC93BA
:100830008FBFDF91CF911F910895DE2BF8CFCF931B
:10084000DF9390E0FC01E955FA4F249188579A4FC5
:10085000FC0184918823D1F090E0880F991FFC015E
:10086000E459FA4FA591B491FC01E658FA4FC591AD
:10087000D49161110EC09FB7F8948C91E22FE0954E
:100880008E238C932881E223E8839FBFDF91CF9151
:1008900008958FB7F894EC91E22BEC938FBFF6CFCD
:1008A0003FB7F8948091090690910A06A0910B0633
:1008B000B0910C0626B5A89B05C02F3F19F00196F4
:1008C000A11DB11D3FBFBA2FA92F982F8827BC01AA
:1008D000CD01620F711D811D911D42E0660F771FD2
:1008E000881F991F4A95D1F708958F929F92AF92D2
:1008F000BF92CF92DF92EF92FF924B015C010E9478
:1009000050046B017C010E9450046C197D098E0912
:100910009F09683E734081059105A8F321E0821A82
:100920009108A108B10888EEC80E83E0D81EE11C2A
:10093000F11C81149104A104B10429F7FF90EF90F8
:10094000DF90CF90BF90AF909F908F90089540918F
:100950006605509167052091640530916505421741
:100960005307B4F49091E8009570E1F39091E8009A
:1009700092FD19C08093F100809166059091670502
:1009800001968F739927892B19F48EEF8093E800D5
:100990008091660590916705019690936705809315
:1009A000660581E0089580E00895EF92FF920F932D
:1009B0001F93CF93DF93F82E192FE62E042F81E09B
:1009C000860F880F0E94A70483E00E94A704CF2D02
:1009D000D12FEC0EFD2EF11CCE15DF05B9F007FF6F
:1009E00013C0FE0184910E94A704182F80E00E948A
:1009F000A704812321968111EFCFDF91CF911F9121
:100A00000F91FF90EF9008958881EDCF81E0F5CFB1
:100A1000DF92EF92FF920F931F93CF93DF93D82E25
:100A20008A01EB017B01E40EF51ECE15DF0559F0BE
:100A3000D7FE12C0FE0184910E94A7042196811165
:100A4000F4CF0FEF1FEFC801DF91CF911F910F91EE
:100A5000FF90EF90DF9008958881EECF2FB7F89444
:100A600087708093E9009091E800892F807295FF4C
:100A700004C09091F20080E4891B2FBF08957F92FB
:100A80008F929F92AF92BF92CF92DF92EF92FF929E
:100A90000F931F93CF93DF93C82E8B017A01809120
:100AA0000E06811110C08FEF9FEFDF91CF911F9144
:100AB0000F91FF90EF90DF90CF90BF90AF909F90FD
:100AC0008F907F90089580916A0580FF05C0809186
:100AD000E00082608093E000CE2DDF2DD12C8AEFE4
:100AE000B82E8C2D8770982E8C2D8072882E8C2D90
:100AF0008074782E9AE3A92E209719F4DD2009F44A
:100B000052C08C2D0E942E0581110AC0BA94BB20C0
:100B100051F261E070E080E090E00E947504ECCF5B
:100B20008C171D0611F00CF08C2F9FB7F894909243
:100B3000E9002091E80025FD02C09FBFDDCF282FEE
:100B400030E0C21BD30B882029F08150A0F0109216
:100B5000F100FBCFF801C7FC0AC0815050F0419171
:100B60004093F100FACF44914093F10031968150C7
:100B7000D0F7020F131FDD2021F0A092E800D12C46
:100B8000DCCF8091E80085FD07C0A092E800DD245D
:100B9000D394209791F2F3CF209779F6772069F2DA
:100BA000A092E800CACF5D9884E680936905C701EA
:100BB0007CCF615030F02091F100FC012083019640
:100BC000F8CF289884E680930D06089580915C05FF
:100BD00081110DC082E08093580584E0809359050F
:100BE00010925B0510925A0581E080935C0588E5C0
:100BF00095E00895EF92FF921F93CF93DF931F929A
:100C0000CDB7DEB77C018091700681112AC011E05A
:100C1000109363061093640689E696E09093660647
:100C20008093650610926806109267068FE494E040
:100C30009093600680935F0610926B0610926A068E
:100C400010926D0610926C0610936E0610936F064C
:100C500081EC809369060E94E6050E94350310939B
:100C6000700682E0898341E050E0BE016F5F7F4FF4
:100C7000809162060E943F0597FD08C08091620640
:100C800048E050E0B70180640E943F050F90DF917B
:100C9000CF911F91FF90EF9008950F931F93CF93E3
:100CA000DF931F92CDB7DEB782E0898342E450E044
:100CB00062E874E080E80E9408050E94E605DC0115
:100CC00012960D911C910115110589F0D801ED9135
:100CD000FC910280F381E02DBE016F5F7F4FC80160
:100CE000099597FD04C0F80100851185ECCF898135
:100CF0000F90DF91CF911F910F910895CF93DF93C4
:100D0000EC0180910B01882331F083E00E943F05C4
:100D10001816190634F081E090E09B838A8380E006
:100D200090E0DF91CF910895CF93DF931F92CDB7DD
:100D3000DEB76983DC01ED91FC910280F381E02D47
:100D400041E050E0BE016F5F7F4F09950F90DF914A
:100D5000CF91089583E08093E9008091F200882389
:100D600019F08AE38093E800089583E00E942E053D
:100D700090E00895CF93DF931F92CDB7DEB7FC01CB
:100D80008485958597FD08C02FEF3FEF3587248731
:100D90000F90DF91CF910895CE0101960E947B03C1
:100DA000019719F4898190E0F3CF8FEF9FEFF0CF97
:100DB0000F931F93CF93DF931F92CDB7DEB78C01B4
:100DC000FC018485958597FF0BC0CE0101960E949A
:100DD0007B03019771F4898190E0F80195878487FE
:100DE000F801848595850F90DF91CF911F910F9128
:100DF00008958FEF9FEFF1CFFC018485958597FDD6
:100E00000BC09FB7F89482E08093E9008091F200D4
:100E10009FBF90E0019608959FB7F89482E0809379
:100E2000E9008091F2009FBF90E00895DC01FB0192
:100E300012962C911297848195812817190641F4F6
:100E400091818081813A31F49D7F81E0913009F078
:100E500080E008958132E1F79B3029F482811F966A
:100E60008C9381E008959A3099F7828150968C9303
:100E7000F8CFDC01FB0188E4808389E4818384E48A
:100E800082831D969C911D979F709F5B93831D96F7
:100E90008D919C9124E0969587952A95E1F78F7026
:100EA0008F5B848385E00895EF92FF920F931F93E9
:100EB000CF93DF93FB012081213871F5238122320A
:100EC00059F5DC0112964C912481358142171306A5
:100ED00019F5EC010B851C85F12CE12C0115110590
:100EE00089F0F801448155816281738180E80E9414
:100EF00008058F3F980749F0E80EF91ED8010D91BB
:100F00001C91ECCF81E08F87C701DF91CF911F91BA
:100F10000F91FF90EF90089590E080E0F6CFCF938F
:100F2000DF93CDB7DEB769970FB6F894DEBF0FBE7B
:100F3000CDBFFC01DB018C918F5F8C939E012D5FF7
:100F40003F4F8DE0D9011D928A95E9F729E0298369
:100F500084E08A8391E09D8383E08E832A8721E267
:100F60002B879C879D879F8722E2288B27E02B8BEE
:100F700025E02C8B8E8B20E430E0388F2F8B998FDF
:100F800082818B8395858685998B8A8B8381806806
:100F90008D8B49E150E0BE016F5F7F4F80E00E9482
:100FA000080569960FB6F894DEBF0FBECDBFDF917E
:100FB000CF91089590910206983169F0E92FF0E001
:100FC000EE0FFF1FE453FA4F808361839F5F90937E
:100FD000020681E0089580E00895CF92DF92EF92BB
:100FE000FF920F931F93CF93DF936C01EB017B0173
:100FF000E40EF51E10E000E0CE15DF0581F06991EA
:101000006D30D1F3D601ED91FC910190F081E02D8E
:10101000C6010995892B19F00F5F1F4FEDCFC8014D
:10102000DF91CF911F910F91FF90EF90DF90CF90C4
:101030000895EF92FF921F93CF93DF93EC01162F49
:10104000E8E7E60F683880F4E62FF0E067FF4FC06E
:10105000E058F10921E030E001C0220FEA95EAF7FB
:101060008C81822B8C83E0E08E818E17D9F08F816A
:10107000E817C1F08885E817A9F08985E81791F08D
:101080008A85E81779F08B85E81761F0DE011696FE
:1010900090E080E02D9121114EC08C0F9D1FDC014E
:1010A0001696EC93CE0104960E94FA05EE24E39482
:1010B000F12C183838F11858DE0186E0112341F080
:1010C00016969C911697191303C016961C921697A4
:1010D000815011968111F2CFCE0104960E94FA053B
:1010E000C701DF91CF911F91FF90EF900895EC5AC7
:1010F000FC4FE491E11118C081E090E09B838A836A
:10110000F12CE12CE12FF0E017FF21C0E058F109AC
:1011100081E090E001C0880FEA95EAF780959C8114
:1011200089238C8310E0C8CFE7FF9ECF8C8182603B
:101130008C83EF7799CF01968630910509F0AACF7D
:1011400081E090E09B838A83F12CE12CB2CFEC5AB2
:10115000FC4F1491112309F4C3CF17FFADCF8C813D
:101160008D7F8C831F77A8CF089590E080E008954D
:10117000CF93DF93FC0101900020E9F73197AF0195
:10118000481B590BBC018FE096E00E947E06EC01E3
:1011900042E050E063E674E08FE096E00E947E0655
:1011A0008C0F9D1FDF91CF910895CF92DF92EF9228
:1011B000FF928091540590915505A0915605B091EC
:1011C00057050196A11DB11D8093540590935505B7
:1011D000A0935605B09357058FB7F894C0900506B5
:1011E000D0900606E0900706F09008068FBFC092E8
:1011F0005005D0925105E0925205F092530580912E
:101200004C0590914D05A0914E05B0914F05805E23
:10121000914BAF4FBF4F8C159D05AE05BF050CF030
:101220004EC020915405309155054091560550917E
:101230005705A8EEB3E00E94701120E23EE440E0C2
:1012400050E00E944B113F932F93C701B60128EE47
:1012500033E040E050E00E944B115F934F933F9387
:101260002F9386E694E09F938F938AE795E09F9370
:101270008F930E94B3118AE795E00E94B80880918D
:10128000500590915105A0915205B091530580935E
:101290004C0590934D05A0934E05B0934F051092C9
:1012A00054051092550510925605109257058DB7AA
:1012B0009EB70A960FB6F8949EBF0FBE8DBFECE0A6
:1012C000F1E013821282749694E0EC32F907C9F7C8
:1012D000FF90EF90DF90CF9008952F923F925F9212
:1012E0006F927F928F929F92AF92BF92CF92DF9236
:1012F000EF92FF920F931F93CF93DF9300D01F9233
:10130000CDB7DEB760E08EE00E94F10361E08EE0D1
:101310000E94F1038FB7F89480900506909006061E
:10132000A0900706B09008068FBF2CE031E03B8309
:101330002A8310E000E097EB292E95E0392E29EA68
:10134000622E24E0722E3AE7E32E35E0F32E4DE8CC
:10135000C42E44E0D42E61E08FE00E94F103E6ED5C
:10136000F5E08491F101F491F983E8E9F5E0549016
:10137000552081F081110E94A503E52DF0E0EE0FCC
:10138000FF1FEC52FC4FA591B4919C91F9819F23D2
:1013900081E009F480E081708983EA81FB818083A8
:1013A00060E08FE00E94F103EA81FB8184819581F6
:1013B000A681B781B501A401481B590B6A0B7B0BB1
:1013C00080859185A285B38584179507A607B70701
:1013D0000CF057C0F981F11119C0EA81FB818181BC
:1013E0008823A1F081E0828384869586A686B786CD
:1013F0001F930F93DF92CF92FF92EF920E94B3114F
:101400000F900F900F900F900F900F90EA81FB813B
:101410008081882331F18181811123C081E0838320
:10142000808A918AA28AB38A84859585A685B785A4
:10143000A5019401281B390B4A0B5B0BDA01C9018A
:10144000BF934F939F932F931F930F937F926F920E
:10145000FF92EF920E94B3110FB6F894DEBF0FBE59
:10146000CDBFEA81FB818281811103C08381882302
:1014700041F0EA81FB8184829582A682B7828081D5
:1014800081830F5F1F4F2A813B812C5E3F4F3B833F
:101490002A830832110509F05ECF3091B0023983FA
:1014A0008091C402882309F43FC060E082E00E947A
:1014B000F10361E083E00E94F10349814423D1F10B
:1014C00060E085E00E94F10361E087E00E94F103A3
:1014D00080916D058823A1F160E089E00E94F1030D
:1014E00061E088E00E94F10380916C05882371F12E
:1014F00060E081E00E94F10361E080E00F900F90D6
:101500000F90DF91CF911F910F91FF90EF90DF909F
:10151000CF90BF90AF909F908F907F906F905F9093
:101520003F902F900C94F10361E082E00E94F10360
:1015300060E0C0CF61E085E00E94F10360E0C5CFCC
:1015400061E089E00E94F10360E0CBCF61E081E0DF
:101550000E94F10360E0D1CFCF92DF92FF920F9310
:101560001F93CF93DF93CDB7DEB76E970FB6F89486
:10157000DEBF0FBECDBFF82E8150990B9C01220F0C
:10158000331FF901EE5CFB4F1491F901ED5CFB4F49
:101590000491F901EE51FC4F65917491CE010196D1
:1015A0006C010E94441162ED74E08AE795E00E94AC
:1015B000AC11DF92CF921F92FF928DED94E09F933A
:1015C0008F938AE795E09F938F930E94B3118AE7E8
:1015D00095E00E94B8080FB6F894DEBF0FBECDBFED
:1015E00080910206853160F460E0812F0E94DA0765
:1015F000602F812F0E94DA0760E0812F0E94DA07B6
:101600006E960FB6F894DEBF0FBECDBFDF91CF91BF
:101610001F910F91FF90DF90CF9008951F920F922E
:101620000FB60F9211242F933F938F939F93AF93F5
:10163000BF938091050690910606A0910706B09190
:1016400008063091040623E0230F2D3758F5019644
:10165000A11DB11D209304068093050690930606F4
:10166000A0930706B09308068091090690910A0698
:10167000A0910B06B0910C060196A11DB11D80939F
:10168000090690930A06A0930B06B0930C06BF912F
:10169000AF919F918F913F912F910F900FBE0F901F
:1016A0001F90189526E8230F0296A11DB11DD2CFD9
:1016B0001F920F920FB60F9211248F939F938091D8
:1016C000E1009091E100937F9093E10083FF0FC0D0
:1016D0001092E90091E09093EB001092EC0092E3FD
:1016E0009093ED0010920E0698E09093F00082FF28
:1016F00022C093E09093E9009091F200992319F0B1
:101700009AE39093E80090916905992341F09091B4
:101710006905915090936905911101C05D9A90916E
:101720000D06992341F090910D06915090930D066E
:10173000911101C0289A84FF18C08091E2008E7E2A
:1017400081608093E2008091E1008F7E8093E100D0
:1017500080916A058E7E806180936A059F918F914A
:101760000F900FBE0F901F90189580FFF7CF8091BC
:10177000E2008E7E80618093E2008091E1008E7EA7
:101780008093E10080916A058E7E8160E5CF1F9293
:101790000F920FB60F921124CF92DF92EF92FF9229
:1017A0000F931F932F933F934F935F936F937F9369
:1017B0008F939F93AF93BF93EF93FF93CF93DF9359
:1017C000CDB7DEB76C97DEBFCDBF1092E900809138
:1017D000E80083FF25C068E0CE0145960E94D90548
:1017E00082EF8093E8008D8987FF39C09091E800EF
:1017F00090FFFCCF982F907609F034C19E894F89D5
:10180000588D2F89F88C911131C0803861F5809105
:101810006B058093F1001092F1008EEF8093E80049
:101820006C960FB6F894DEBF0FBECDBFDF91CF919F
:10183000FF91EF91BF91AF919F918F917F916F91A8
:101840005F914F913F912F911F910F91FF90EF90DA
:10185000DF90CF900F900FBE0F901F9018959EEFC6
:101860009093E800C7CF1092F100D5CF913059F492
:101870008111D3CF4130510581F680916B058D7F69
:1018800080936B05CACF933049F48111C6CF4130A4
:10189000510519F680916B058260F2CF953041F4C5
:1018A0008091E80080FFFCCF20682093E300B5CF53
:1018B000963009F0A9C00B8D1C8D22E01092E90032
:1018C0001092670510926605F2122EC010926505FF
:1018D000109264050E944D061F8299E09983FA8256
:1018E00091E09E8390EA98879AEF99872091660508
:1018F00030916705275F3F4F3C832B838D83109288
:10190000E900109267051092660510936505009333
:10191000640549E050E0BE016F5F7F4F80E00E94A8
:1019200008050E944D0679CF109365050093640564
:101930000E94E605DC0112960D911C91011511051E
:1019400009F451C1D801ED91FC910480F581E02D9D
:10195000BE016B5E7F4FC8010995009709F03EC13B
:10196000F80100851185EACFF3E0FF120EC08F89E0
:10197000882309F440C0823061F440E869E080EED9
:1019800094E00E94D504811148CF81E28093EB005E
:1019900047CF813029F440E865E08AED94E0F1CF4B
:1019A000833099F70E94E605DC011296ED90FC90D9
:1019B0008E010F5F1F4F6801E114F10479F0D70128
:1019C000ED91FC910680F781E02DB801C7010995E2
:1019D000080F111DF701E084F184EECFD8011C92AD
:1019E000F60101900020E9F73197BF016C197D09DC
:1019F00040E0C601C6CF64EC74E0FB01449150E0C6
:101A000080E80E94080509CF973009F4BECF9830CE
:101A100021F481E08093F10000CF993009F0FDCEF0
:101A2000837009F0B2CFEDE2F4E081E031E096E3BB
:101A30002191222371F08093E9003093EB00DF01C4
:101A400011972C912093EC009093ED008F5F8730DD
:101A500079F78EE78093EA001092EA008F898093ED
:101A60000E06DBCE8B8D9C8D1092E90010926705DF
:101A7000109266059093650580936405898D8111A8
:101A800092C08E899D89913A49F4813209F07DCFC7
:101A900047E050E064E071E080E0B3CF913209F0BC
:101AA00074CF833269F48F89988DB0E0A0E0809381
:101AB000000190930101A0930201B0930301ADCE08
:101AC000803269F48091E80082FFFCCF67E084E017
:101AD00091E00E94D9058BEF8093E8009ECE823280
:101AE00009F09BCE8F8980930B01EEEFFFE7859184
:101AF00094918B3F9C4D51F1E0E0F8E0809104011E
:101B000090910501A0910601B0910701803B94409E
:101B1000A105B105F1F480910B0180FD1AC0EE3FE3
:101B20008AE0F80789F587E797E7918380838091BA
:101B300060008093680588E19BE00FB6F894A89553
:101B4000809360000FBE9093600067CEEEEFFAE0E6
:101B5000D5CF808191818737974709F05ECEA895D0
:101B60008091600088618093600080916805809317
:101B70006000EE3F2AE0F20789F08091FE0A909122
:101B8000FF0A9183808349CE8081918187379807AE
:101B900051F29093FF0A8093FE0AC5CF1092FF0A7C
:101BA0001092FE0A3ACE0E94E605DC0112960D91D3
:101BB0001C910115110509F4E8CED801ED91FC91B5
:101BC0000190F081E02DBE016B5E7F4FC801099549
:101BD000811123CEF80100851185EBCF1816190667
:101BE0000CF41BCED2CEF1E0FF12BECE68EC74E056
:101BF00004CFCF93109212061092110688EE93E054
:101C0000A0E0B0E08093130690931406A09315060D
:101C1000B09316068DE394E09093100680930F0620
:101C20008FEF9FEF90931C0680931B0610928906FE
:101C3000109288068BE594E0909387068093860641
:101C400080917E06811113C0109279061092780659
:101C500085EE95E090937B0680937A068FE290E084
:101C600090937D0680937C0681E080937E06809130
:101C7000700681112AC0C1E0C0936306C093640658
:101C800089E696E090936606809365061092680652
:101C9000109267068FE494E09093600680935F064D
:101CA00010926B0610926A0610926D0610926C06E6
:101CB000C0936E06C0936F0681EC809369060E9404
:101CC000E6050E943503C0937006E0916A06F09124
:101CD0006B063097B9F488E796E090936B06809393
:101CE0006A0680916C0690916D0620917C06309179
:101CF0007D06820F931F90936D0680936C06CF91A3
:101D00000895FC01808191810097D9F788E796E0DA
:101D100091838083E6CFCF93DF93CDB7DEB7629711
:101D20000FB6F894DEBF0FBECDBF789484B5826045
:101D300084BD84B5816084BD85B5826085BD85B56F
:101D4000816085BD80916E00816080936E001092ED
:101D50008100809181008260809381008091810068
:101D600081608093810080918000816080938000F9
:101D700080919100826080939100809191008160B8
:101D80008093910080919000816080939000809179
:101D9000C10084608093C1008091C1008260809303
:101DA000C1008091C10081608093C1008091C30017
:101DB00081608093C3008091C00082608093C000E6
:101DC0008091C20081608093C20080917A0084601B
:101DD00080937A0080917A00826080937A0080916B
:101DE0007A00816080937A0080917A008068809385
:101DF0007A0010920E0610926B0510926A0580917F
:101E0000D70081608093D70080EA8093D80089B59D
:101E1000806189BD89B5826089BD09B400FEFDCFAE
:101E200061E070E080E090E00E9475048091D8004D
:101E30008F7C80618093D8008091E000807F8093C8
:101E4000E0008091E1008E7E8093E1008DE0809340
:101E5000E200559A209A61E082E00E941F0461E04E
:101E600083E00E941F0461E085E00E941F0461E09E
:101E700087E00E941F0461E089E00E941F0461E086
:101E800088E00E941F0461E081E00E941F0461E07D
:101E900080E00E941F048FEF9FEF90931C068093B9
:101EA0001B0661E08EE00E941F0461E08FE00E944B
:101EB0001F0460E080E10E941F04A0E1B5E084E11E
:101EC00045E050E060E070E0EC918E9FF00111245D
:101ED000E45FFE4F4087518762877387129625E043
:101EE000A633B20789F70E946D090E94D50864E6FF
:101EF00070E080E090E00E9475048E010F5F1F4F3C
:101F0000F4E13F2ECE010B963C01AAE74A2EA5E054
:101F10005A2E222423940E946D09F12CE12CF70102
:101F2000E05FFA4FC490F701EF5EFA4FB490F7010B
:101F3000E651FB4F65917491C8010E94441196E1EE
:101F4000C9122AC18091C702882311F0E5E2BE2E92
:101F50009091C602992309F494C176E2B72E8B2D95
:101F60000E94AC0A60E080E00E94DA0720E6A22E20
:101F700025E0B22E3EE6C32E35E0D32E44E5842E76
:101F800045E0942EF12CE12CF50184913196E491F9
:101F900090E0389ED001399EB00D1124A45FBE4F51
:101FA00012962C911297211105C013962C91222381
:101FB00009F43BC0389ED001399EB00D1124A45FB6
:101FC000BE4F3E9EF0011124E45FFE4F9C91808144
:101FD00098132FC181E0F601808394E0E3E3F4E0FD
:101FE000D30101900D929A95E1F7188A1F868130EE
:101FF00029F462E075E0C3010E94AC11F40165911F
:102000007491C8010E9444117F926F921F930F93A5
:1020100026E035E03F932F935F924F920E94B311D9
:102020000FB6F894DEBF0FBECDBFF60180819701D9
:102030002F5F3F4F3A8B298B882321F13AE0239F72
:10204000902D11249F5FE114F10409F4F4C0E5E040
:10205000EE16F10409F4F3C030E020E0F901EA5C87
:10206000FA4FE491E913F3C0F901E80FF11DEA5CBE
:10207000FA4F84910E94AC0A60E080E00E94DA0787
:10208000F6011082F2E0AF0EB11C22E0C20ED11CAC
:1020900032E0830E911CE988FA8886E0E816F104A4
:1020A00009F072CF0E94D5088FB7F894C09005064A
:1020B000D0900606E0900706F09008068FBF80914A
:1020C0000306811105C090910206992309F45CC0B2
:1020D0004091FE055091FF05609100067091010648
:1020E0004C155D056E057F050CF04EC0E82FF0E045
:1020F000EE0FFF1FE453FA4F90819093CB0521819F
:102100002093CA058F5F809303061F922F931F921F
:102110009F93FF92EF92DF92CF9288E195E09F9399
:102120008F935F924F920E94B3118AE795E00E94CD
:10213000B80888E0F80111928A95E9F79091CB05EB
:102140000FB6F894DEBF0FBECDBF8091CA059111C6
:1021500085C0811183C0C8010E94FA05C092FE05A6
:10216000D092FF05E0920006F09201068AE395E026
:102170000E94B8089091030680910206981304C04B
:10218000109202061092030680E090E0892B09F479
:10219000C2CE0E940000BDCEE1E2CE120AC0809104
:1021A000A3038823D9F180916D05822580936D0565
:1021B000DDCEF8E0CF120AC08091AF01882371F123
:1021C00080916C05822580936C05D0CE24E1C212EB
:1021D00025C08091B00263E2B62E811102C054E2A4
:1021E000B52ED12C3C9CF0013D9CF00D1124E45FF8
:1021F000FE4F8281882319F08B2D0E94AC0A3C9CF3
:10220000F0013D9CF00D1124E45FFE4F8381882393
:1022100039F060E080E00E94DA0702C0B110E1CF3F
:1022200032E0E30EF11C86E2E816F10409F077CE05
:102230009DCE82E0D0CE20916D05920F0DCF2091E2
:10224000B002211101C09FE320916C05F6CF2D5FF4
:102250003F4F2E31310509F001CF12CF99838B8387
:10226000C8010E94FA053EE1C30ED11CE11CF11C1D
:10227000C092FE05D092FF05E0920006F0920106A2
:1022800079CF81116CCE72CEFB01DC0105900D92ED
:102290000020E1F70895052E97FB1EF400940E949C
:1022A000621157FD07D00E947B1107FC03D04EF44A
:1022B0000C94621150954095309521953F4F4F4FAA
:1022C0005F4F089590958095709561957F4F8F4FE2
:1022D0009F4F0895EE0FFF1F0590F491E02D099494
:1022E0000E949D11A59F900DB49F900DA49F800DFD
:1022F000911D11240895A1E21A2EAA1BBB1BFD01FA
:102300000DC0AA1FBB1FEE1FFF1FA217B307E407D4
:10231000F50720F0A21BB30BE40BF50B661F771F2C
:10232000881F991F1A9469F760957095809590950C
:102330009B01AC01BD01CF010895A29FB001B39FE5
:10234000C001A39F700D811D1124911DB29F700DBE
:10235000811D1124911D0895FB01DC0101900D9256
:102360000020E1F70895AEE0B0E0E9EBF1E10C9474
:1023700062140D891E8986E08C831A8309838FEF8E
:102380009FE79E838D83AE01475E5F4F6F89788D97
:10239000CE0101960E94D6112F813885020F131F9E
:1023A000F80110822E96E4E00C947E14ABE0B0E0CD
:1023B000ECEDF1E10C9454147C013B018A01FC0129
:1023C00017821682838181FFC8C1CE0101965C010C
:1023D000F7019381F30193FD859193FF81913F0173
:1023E000882309F453C1853239F493FD859193FF15
:1023F00081913F01853229F4B70190E00E94C61314
:10240000E7CF912C212C312CFFE1F31538F08B32E2
:1024100011F190F4803209F1833229F137FC3CC08C
:1024200020ED280F2A3050F536FE20C08AE0989E15
:10243000200D1124922E06C08D3291F0803371F759
:10244000689430F8F30193FD859193FF81913F01EA
:102450008111DACF21C0689431F8689432F8F2CF54
:10246000689433F8EFCF689434F8ECCFEAE02E9E0E
:10247000200D1124222E689435F8E4CF8E3229F4F1
:1024800036FC04C1689436F8DDCF8C3619F46894B4
:1024900037F8D8CF8836B1F2982F9F7D9554933076
:1024A000E0F08336A1F18337C1F1833509F063C0D1
:1024B0002801F2E04F0E511CF801C080D180692D37
:1024C00070E036FC02C06FEF7FEFC6010E94B013D0
:1024D0004C01689437F882010AC00C5F1F4FFFE37C
:1024E000F98388248394912C6501E89437F833FEAE
:1024F0002DC0522C8114910471F5552009F468CF38
:10250000B70180E290E00E94C6135A94F6CFF8011A
:10251000808189830E5F1F4FE4CF2801F2E04F0EC8
:10252000511CF801C080D180692D70E036FC02C0DA
:102530006FEF7FEFC6010E94BB134C018201D5CF24
:10254000B70180E290E00E94C6132A94281419046F
:1025500009F0B0F7CECFF60137FC859137FE8191B7
:102560006F01B70190E00E94C61351105A94F1E038
:102570008F1A9108BFCF843619F0893609F077C0D9
:10258000F80137FE6BC060817181828193810C5F9D
:102590001F4FF32DFF763F2E97FF09C09095809532
:1025A000709561957F4F8F4F9F4F689437F82AE061
:1025B00030E0A5010E94F613C82ECA188C2C432CBB
:1025C00036FE0CC0E89440F8C91440F434FE05C04F
:1025D00032FC03C0F32DFE7E4F2E892C44FE95C0A5
:1025E000FE01EC0DF11D8081803309F087C0242DA0
:1025F000297E422E842D8870582E43FC95C040FEC3
:102600008FC09C2C821418F42C0C922C981844FE29
:1026100091C0B70180E390E00E94C61342FE09C05A
:1026200088E790E041FE02C088E590E0B7010E9493
:10263000C613C91408F48AC0CA94D12C9FEFC91AD2
:10264000D90ACA0CDB1CF60182916F01B70190E038
:102650000E94C613AC14BD04B1F74FCF60817181E5
:10266000072E000C880B990B0E5F1F4F92CFD32CB7
:10267000E894D4F82AE030E0853739F1232D297F1A
:10268000D22E8F3601F148F48835A9F0F701868102
:1026900097812B96E2E10C947014803749F08837CB
:1026A000A9F7D4FE02C06894D2F820E130E00DC052
:1026B0006894D4F8F6CF34FE03C0822F8660D82EFB
:1026C00020E132E002C028E030E0F801D7FE0FC080
:1026D00060817181828193810C5F1F4FA5010E94EF
:1026E000F613C82ECA183D2CE89437F867CF6081DE
:1026F000718190E080E00E5F1F4FF0CF42FC02C07E
:10270000839478CF8394839475CF842D867809F44D
:1027100071CFF6CFB70180E290E00E94C613839498
:102720008214C0F3512C73CF522C5818821408F421
:102730006ECFF8CF842D867809F47BCF8BE241FEF3
:1027400080E247FC8DE2B70190E071CFB70180E3F2
:1027500090E00E94C6139A946CCF8FEF9FEF99CFB1
:10276000FC010590615070400110D8F7809590955C
:102770008E0F9F1F0895FC01615070400190011061
:10278000D8F7809590958E0F9F1F08950F931F93F4
:10279000CF93DF93182F092FEB018B8181FD09C0A7
:1027A0001FEF0FEF812F902FDF91CF911F910F918E
:1027B000089582FF14C02E813F818C819D8128174E
:1027C00039073CF4E881F981CF0101969983888328
:1027D00010838E819F8101969F838E83E3CFE8854E
:1027E000F985812F0995892BA1F3DACFFA01AA2760
:1027F000283051F1203181F1E8946F936E7F6E5F44
:102800007F4F8F4F9F4FAF4FB1E03ED0B4E03CD0F1
:10281000670F781F891F9A1FA11D680F791F8A1FD4
:10282000911DA11D6A0F711D811D911DA11D20D03B
:1028300009F468943F912AE0269F11243019305DF5
:102840003193DEF6CF010895462F4770405D4193E6
:10285000B3E00FD0C9F7F6CF462F4F70405D4A3333
:1028600018F0495D31FD4052419302D0A9F7EACFFB
:10287000B4E0A6959795879577956795BA95C9F72A
:1028800000976105710508959B01AC010A2E06941D
:102890005795479537952795BA95C9F7620F731FD6
:1028A000841F951FA01D08952F923F924F925F9213
:1028B0006F927F928F929F92AF92BF92CF92DF9250
:1028C000EF92FF920F931F93CF93DF93CDB7DEB7B5
:1028D000CA1BDB0B0FB6F894DEBF0FBECDBF099449
:1028E0002A88398848885F846E847D848C849B84A0
:1028F000AA84B984C884DF80EE80FD800C811B81AE
:10290000AA81B981CE0FD11D0FB6F894DEBF0FBEDC
:0A291000CDBFED010895F894FFCF4C
:10291A00FFFFFFFF00E100000000000001010000CE
:10292A00000000000000000000000000000000009D
:10293A00010100000000000000000000000000008B
:10294A00000000000101000000000000000000007B
:10295A00000000000000000001010000000000006B
:10296A00000000000000000000000000010100005B
:10297A00000000000000000000000000000000004D
:10298A00010100000000000000000000000000003B
:10299A00000000000101000000000000000000002B
:1029AA00000000000000000001010000000000001B
:1029BA00000000000000000000000000010100000B
:1029CA0000000000000000000000000000000000FD
:1029DA0001010000000000000000000000000000EB
:1029EA0000000000010100000000000000000000DB
:1029FA0000000000000000000101000000000000CB
:102A0A0000000000000000000000000001010000BA
:102A1A0000000000000000000000000000000000AC
:102A2A00010100000000000000000000000000009A
:102A3A00000000000101000000000000000000008A
:102A4A00000000000000000001010000000000007A
:102A5A00000000000000000000000000010100006A
:102A6A00000000000000000000000000000000005C
:102A7A00010100000000000000000000000000004A
:102A8A00000000000101000000000000000000003A
:102A9A00000000000000000001010000000000002A
:102AAA00000000000000000000000000010100001A
:102ABA00000000000000000000000000000000000C
:102ACA0001010000000000000000000000000000FA
:102ADA0000000000010100000000000000000000EA
:102AEA0000000000000000000101000000000000DA
:102AFA0000000000000000000000000001010000CA
:102B0A0000000000000000000000000000000000BB
:102B1A0001010000000000000000000000000000A9
:102B2A000000000001010000000000000000000099
:102B3A000000000000000000010100000000000089
:102B4A000000000000000000000000000101000079
:102B5A00000000000000000000000000000000006B
:102B6A000101000000000000000000000000000059
:102B7A000000000001010000000000000000000049
:102B8A000000000000000000010100000000000039
:102B9A000000000000000000000000000101000029
:102BAA00000000000000000000000000000000001B
:102BBA000101000000000000000000000000000009
:102BCA0000000000010100000000000000000000F9
:102BDA0000000000000000000101000000000000E9
:102BEA0000000000000000000000000001010000D9
:102BFA0000000000000000000000000000000000CB
:102C0A0001010000000000000000000000000000B8
:102C1A0000000000010100000000000000000000A8
:102C2A000000000000000000010100000000000098
:102C3A0000000000000000000000000000C18081C8
:102C4A000000002D2D3E0000000000000094067ECA
:102C5A0006B506AA06FC06BA06D806000000001643
:102C6A00078F0754073907000000001908ED07B558
:102C7A0008B4080D0A00205B543A256C6420736579
:102C8A00635D2041766572616765207363616E20BA
:102C9A0070657220736563203D20256400496E705B
:102CAA007574206E756D6265723A25642052616989
:102CBA0073696E67466C616700496E707574206E41
:102CCA00756D6265723A25642046616C6C696E673F
:102CDA00466C6167202028543D2564206D73656326
:102CEA005D00313233343536373839300050726549
:102CFA00737320436F6D6D616E6420436F64653A30
:102D0A00256920436F6D62696E6174696F6E3A2539
:102D1A0073003C2D2D00456E636F6465723A25730E
:102D2A00205B202573205D00205B6D7365633D2564
:102D3A006C64205D20204D6F646966696572733A20
:102D4A002564204B65793A25640052656C65617388
:0C2D5A006520616C6C206B6579730000D3
:00000001FF
